:100000000C9439030C9480030C9480030C948003AB
:100010000C9480030C9480030C9480030C94800354
:100020000C9480030C9480030C942B290C94FD29D0
:100030000C94FE1F0C9480030C9480030C9480039A
:100040000C9480030C9480030C9480030C94800324
:100050000C9480030C944B200C9480030C9480032C
:100060000C9480030C9480030C9480030C94800304
:100070000C9480030C9480030C9480030C948003F4
:100080000C9480030C9480030C9480030C948003E4
:100090000C9480030C9480030C9480030C948003D4
:1000A0000C9480030C9480030C948003530E560E22
:1000B0005E0E630E680E6D0E720E770E7C0E810E54
:1000C000860E8B0E8D0E900E930E960E990E9C0E34
:1000D0009E0EA30E4615461578157815C515E31521
:1000E00004170417EE15831694169416F4160417C5
:1000F0000417FD16A417A417B617B617AD17B61731
:10010000B617B617A417A417B217B617B617B217B3
:100110006A2A912A892B912A892BDD2A002B892B87
:10012000572B662B35001E001F00200021002200E7
:10013000230024002500260027002D002E000000AB
:100140002A002B00000014001A00080015001700F8
:100150001C0018000C00120013002F0030003100AA
:100160002900000004001600070009000A000B0027
:100170000D000E000F003300340028000000E100E5
:1001800000001D001B0006001900050011001000F2
:100190003600370038000000E5000000E000E20013
:1001A0000000E300000000002C0000000000000040
:1001B000E70001510000E600E40000003A003B00C7
:1001C0003C003D003E003F00400041004200430033
:1001D000440045000000000000000000BD00BE001B
:1001E00000000000000000000000520000000000BD
:1001F00000000000C25C39000000000000000000A8
:10020000000000000000500051004F0000000000FE
:1002100000000000000000000000000000000000DE
:100220000000000000004E004B0000000000000035
:1002300000000000000000000000000000000000BE
:1002400000000000000000000000000000000000AE
:10025000000000000000000000000000000000009E
:10026000000000000000000000000000000000008E
:10027000000000000000000000000000000000007E
:10028000000000000000000000000000000000006E
:10029000000000000000000000000000000000005E
:1002A000000000000000000000000000000000004E
:1002B0000000000000000000BE00BD0000000000C3
:1002C000000000000000000000000000000000002E
:1002D000000000000000000000000000000000001E
:1002E00000000000010032190A00047F3F1F643241
:1002F00014643214783C1E1E140A05222325262875
:10030000292A2C2D2F3032333536383A3B3D3E40AA
:1003100042434547494A4C4E5051535557595A5CF0
:100320005E6062646668696B6D6F71737577797B07
:100330007D7F81838587898A8C8E90929496989A06
:100340009C9E9FA1A3A5A7A8AAACAEAFB1B3B4B61B
:10035000B8B9BBBCBEBFC1C2C3C5C6C7C9CACBCC76
:10036000CDCED0D1D2D2D3D4D5D6D7D7D8D9D9DA49
:10037000DADBDBDBDCDCDCDCDCDDDDDDDDDCDCDCBE
:10038000DCDCDBDBDBDADAD9D9D8D7D7D6D5D4D3E6
:10039000D2D2D1D0CECDCCCBCAC9C7C6C5C3C2C1BB
:1003A000BFBEBCBBB9B8B6B4B3B1AFAEACAAA8A718
:1003B000A5A3A19F9E9C9A98969492908E8C8A89D0
:1003C000878583817F7D7B79777573716F6D6B69AD
:1003D00068666462605E5C5A5957555351504E4C82
:1003E0004A4947454342403E3D3B3A383635333231
:1003F000302F2D2C2A292826252322FFAA7F55407D
:1004000000010101010101010101020202020202D7
:1004100002020203030303030303030404040404AA
:100420000404050505050506060606060707070771
:100430000708080808090909090A0A0A0B0B0B0C26
:100440000C0C0D0D0D0E0E0E0F0F0F1010111111C3
:100450001212131314141515161617171818191944
:100460001A1A1B1B1C1D1D1E1E1F202021222223A9
:100470002424252626272829292A2B2C2D2D2E2FEA
:1004800030313232333435363738393A3B3C3D3E01
:100490003F404142434445464748494A4C4D4E4FF0
:1004A00050515354555658595A5B5D5E5F616264B2
:1004B000656668696B6C6D6F7072737577787A7B3F
:1004C0007D7E8082838587888A8C8E8F9193959696
:1004D000989A9C9EA0A2A3A5A7A9ABADAFB1B3B5B6
:1004E000B7BABCBEC0C2C4C6C9CBCDCFD1D4D6D892
:1004F000DBDDDFE2E4E7E9EBEEF0F3F5F8FAFDFF30
:100500000403300000000A0344005A0036003000A3
:10051000000010034B0042004400460061006E00E2
:10052000730000000403090409023B00020100A05B
:10053000FA09040000010301010009211101000171
:100540002240000705810308000A09040100010395
:1005500000000009211101000122BC0007058203EF
:1005600020000A12011001000000085A4460220114
:10057000000102030105010902A10185020901A18F
:100580000005091901290515002501950575018149
:100590000295017503810105010930093115812595
:1005A0007F95027508810609381581257F950175AB
:1005B000088106050C0A38021581257F950175080A
:1005C0008106C0C005010980A101850319012AB770
:1005D00000150126B700950175108100C0050C09B2
:1005E00001A101850419012AA002150126A0029586
:1005F0000175108100C005010906A10185050507E7
:1006000019E029E715002501950875018102050704
:10061000190029EF1500250195F0750181020508E3
:10062000190129059505750191029501750391013F
:10063000C005010906A101050719E029E7150025F4
:100640000195087501810295017508810105071959
:100650000029FF150026FF00950675088100050892
:1006600019012905950575019102950175039101FF
:10067000C00011241FBECFEFDAE0DEBFCDBF04B64D
:1006800003FE27C080916A0390916B03A0916C03D5
:10069000B0916D038730904BA740B04BD1F41092CE
:1006A0006A0310926B0310926C0310926D0314BED8
:1006B00084B7877F84BF0FB6F894A89580916000B7
:1006C000886180936000109260000FBEE0E0F8E364
:1006D000099511E0A0E0B1E0EAE3FAE502C0059077
:1006E0000D92AC3CB107D9F723E0ACECB1E001C00E
:1006F0001D92AA36B207E1F70E945A260C941B2DD0
:100700000C940000229A2A9A08950E9474060C9470
:10071000820381FF02C02A9801C02A9A0C94EC033C
:1007200081E0089581E008950C94920308950C945B
:1007300096031F93CF93DF9300D000D01F92CDB7C5
:10074000DEB749835A836B833091400289819A8155
:10075000311114C0662359F0222349F00E94DD1C98
:10076000182F682F89819A810E94861C03C00E94DD
:10077000B11C182F69817A81812F04C00E94DD1C71
:1007800069817A810F900F900F900F900F90DF91F9
:10079000CF911F910C945704FC01262F4081518169
:1007A0006281738184810C949903CF93DF93EC0170
:1007B00060E00E94CC03BE01DF91CF910C949703BF
:1007C0000E940F1E811102C00E94C21E0E941E10B4
:1007D0000C9485030C947206089581E008950C949E
:1007E000ED03CF93C82F0E9489038C2F0E94EF0343
:1007F000CF91089508950E9492170E94FA032FEF57
:1008000084E39CE0215080409040E1F700C000006C
:100810000C9471200F931F93CF93DF93EC0161E051
:100820000E94CC038C01BE010E9494038823A9F18D
:10083000BE01C8010E94870F882379F1BE01C8015B
:100840000E94CD10882349F1BE01C8010E940E11FB
:10085000882319F1BE01C8010E9439128823E9F0EA
:10086000BE01C8010E943C0E8823B9F08A8188230A
:1008700069F001158CE5180731F00E3D1C4531F487
:100880000E94C21E0AC00E94FB0307C0CE01DF9176
:10089000CF911F910F910C94900380E0DF91CF9145
:1008A0001F910F91089580E090E0089508952BE442
:1008B000829FC0011124FC012FE0729FE00DF11D09
:1008C0001124E60FF11DEE0FFF1FEC5DFE4F859129
:1008D00094910895880F991FFC01EA51FD4F85916D
:1008E00094910895CF93DF930E9457040E948A0544
:1008F000EC018115904508F041C0C11580E4D8078E
:1009000008F0D1C0C83ED10510F5C03ED10508F0B1
:10091000FDC0C83AD10578F4C53AD10508F0A2C0A7
:10092000C130D10509F4F2C008F4EEC0C430D105DD
:1009300008F0ECC0E9C0CF3BD10508F49BC0C03C37
:10094000D10508F4E1C0CE01805C91099EC0C115BB
:1009500090E2D90758F4C11521E0D20708F0D6C0BB
:10096000C03FD10508F4D0C0D065D0C0C11580E328
:10097000D80708F08EC0CE019F7087C0C11595E5DD
:10098000D90708F043C0C11524E5D20708F0A2C07A
:10099000C11582E5D80708F5C11591E5D90708F01A
:1009A00085C0CE0174E0969587957A95E1F78370BE
:1009B0009C2F937021E030E002C0220F331F9A95E4
:1009C000E2F73C68382BCF70C695C69580E2C89F89
:1009D000E0011124C22BD32B99C09E012370332731
:1009E0008C2F86958695C115D34508F064C0C1E06B
:1009F000D0E002C0CC0FDD1F2A95E2F720E2829FF3
:100A0000C0011124C82BD92BDC6880C0C11529E591
:100A1000D207A0F4C11588E5D80708F060C0C11559
:100A200096E5D90708F070C08C2F0E941E068F71C2
:100A3000C82FD0E0DC2FCC27D06268C0C1152AE5D2
:100A4000D20708F451C0CE0190568115904208F0AB
:100A50005BC08D2F8F710E941E06DD27D0628F71C3
:100A6000D82B54C0C55AD0E0C75ADE4FC881D0E059
:100A7000D0644CC0C85AD0E0CC0FDD1FC55DDE4F3E
:100A80000990D881C02DD46441C00E946A04EC0151
:100A90003DC0CE019927D3FF03C0EC01D86C36C00E
:100AA000EC01D06C33C0DF70D06A30C0DC2FCC27B3
:100AB000C16FD06A2BC0C1E0D0E002C0CC0FDD1FF7
:100AC0002A95E2F720E2829FC0011124C82BD92B7E
:100AD000DA681CC0DC2FCC27C46FD06A17C0DC2FAB
:100AE000CC27C06FD06A12C08C2F8F700E941E0658
:100AF00094E0D695C7959A95E1F7CF70D0E0DC2FBA
:100B0000CC27D069C82B02C0C0E0D0E0CE01DF9175
:100B1000CF9108958238910569F1B0F48133910540
:100B200009F46DC048F48932910509F463C08A3232
:100B3000910509F469C008958533910509F455C0FC
:100B400089339105B9F00895833E910569F138F430
:100B5000803E9105B1F0823E910509F10895863EEF
:100B60009105A9F1873E9105B9F1843E910509F0FF
:100B700064C023C020915B0320FD4FC021FD4DC008
:100B8000089580915B0380FD44C080915C0380FFE9
:100B900044C080915B0384FD42C083EE4DC08091D0
:100BA0005B0382FF38C0F5CF80915B0382FD33C0C9
:100BB00080915C0380FD31C0ECCF80915C0381FFAC
:100BC00032C080915B0384FD2AC087EE35C08091DE
:100BD0005B0383FF26C0F5CF80915B0383FD21C0BB
:100BE00080915C0381FD1FC0ECCF80915B0385FD8C
:100BF0001CC01DC080915B0385FD19C016C080918B
:100C00005B0386FD16C017C080915B0386FD13C091
:100C100010C089E311C082EE0FC080EE0DC080E0ED
:100C20000BC086EE09C084EE07C089E205C085E3EB
:100C300003C08AE201C081E390E0089590915B03D4
:100C400092FF0DC0282F2871283019F4877F846007
:100C500006C0282F2471243011F48B7F886093FF05
:100C60000DC0282F2871283119F4877E846106C0B1
:100C7000282F2471243111F48B7E886120915C032C
:100C800020FF0DC0382F3871383019F4877F81600C
:100C900006C0382F3171313011F48E7F886021FF0A
:100CA0000DC0282F2871283119F4877E816106C074
:100CB000282F2171213111F48E7E886194FD877E69
:100CC0000895E82FF0E0EE0FFF1FE95EFC4F8081F2
:100CD00091810895089580EA8A95F1F7089508951D
:100CE0000C946F060C9470060C946F06CF93DF93F0
:100CF000ABE6B1E040E751E061E070E08D91E82FB4
:100D0000E295EF70F0E021A18F70EB0102C0CC0FF3
:100D1000DD1F8A95E2F7CE019C2F9095922391A337
:100D200092A1892B82A34A175B0741F7ACE5B1E09A
:100D30004BE651E061E070E08D91E82FE295EF70B5
:100D4000F0E021A18F70EB0102C0CC0FDD1F8A956E
:100D5000E2F7CE019C2F9095922391A392A1892B2B
:100D600082A34A175B0741F7EDE0F3E0A7E1B3E0A8
:100D700087E193E0119211921D921D928E179F07A9
:100D8000C9F785E00E945507DF91CF910C94E003ED
:100D90006F927F928F929F92AF92BF92CF92DF928B
:100DA000EF92FF920F931F93CF93DF938BE6C82EA2
:100DB00081E0D82E0DE013E097E1A92E93E0B92E43
:100DC000712C88248394912CF60181916F01C82F96
:100DD000C295CF70D0E099A18F70740101C0EE0C64
:100DE0008A95EAF7892F8E2989A38AA16E2C6094AF
:100DF00086218AA30E946B06ECE5F1E040E050E01A
:100E000020E030E06191A62FA295AF70B0E09096FF
:100E10008C9190E06F7002C0959587956A95E2F786
:100E200080FD08C0C401042E02C0880F991F0A94D7
:100E3000E2F702C080E090E0282B392B4F5F5F4F34
:100E40004F305105F9F689A1682269A28AA1E82AE2
:100E5000EAA2F801808191812817390721F03183B6
:100E6000208381E001C080E0782A0E5F1F4FA0162A
:100E7000B10609F0A9CF272D45E067E173E08DE0C9
:100E800093E00E9456070E94EA03872DDF91CF91DD
:100E90001F910F91FF90EF90DF90CF90BF90AF9098
:100EA0009F908F907F906F9008950895FF920F9379
:100EB0001F93CF93DF93F82E092F162FD72FC42F10
:100EC000222349F081E08093CE010E94302090934C
:100ED000CD018093CC018091CE018823D9F08091FF
:100EE000CC019091CD010E943C20069798F0EF2D07
:100EF000F02FA12FBD2F80E090E04C2F50E0841701
:100F0000950734F4219131912D933D930196F7CFBC
:100F10001092CE01DF91CF911F910F91FF90089514
:100F2000EF92FF920F931F93CF93DF93F62E472FED
:100F3000E82FF0E0711106C0E050FC4F6491762F6D
:100F4000862F72C0272F30E0E050FC4FE4910E2F27
:100F500010E056E0659FC0011124CFEFD0E0BE0144
:100F60000E94D92B5BEA5603C001579F900D1124B4
:100F70008F0D911D8F0D911D982F990F890F7E0157
:100F8000E21AF30AE09ED001E19EB00DF09EB00D92
:100F90001124489FA0011124452F55277E01E41AF2
:100FA000F50AE09EA001E19E500DF09E500D112427
:100FB0007E01E81AF108E29EC001E39E900DF29EC8
:100FC000900D1124892F9927C81BD90BC09FC001F0
:100FD000C19F900DD09F900D11246230710591F04A
:100FE00048F461157105E1F061307105A9F48B2FAA
:100FF000752F19C06430710561F038F066307105E5
:1010000079F00AC0892F7B2F0EC08E2F7B2FE52F02
:101010000AC08E2F792F02C0852F7E2FEB2F03C0A1
:101020008B2F7E2FE92F6E2FDF91CF911F910F9184
:10103000FF90EF9008950895CF93DF93762FE90105
:10104000682F842F0E949007798368838A83DF91B9
:10105000CF91089580912103282F269530E0211506
:10106000310519F48170826005C02B32310524F0FE
:101070008170846580932103089588E090E00C944A
:10108000B42CCF92DF92EF92FF926B017C010E9411
:101090002A08B701A60188E090E0FF90EF90DF906A
:1010A000CF900C94D22CE1E2F3E083E080831182B4
:1010B0008FEF828383831482608171818281938127
:1010C0000C9441088091210380FF02C08695089509
:1010D00080E0089580912503833018F48F5F80931A
:1010E0002503609121037091220380912303909145
:1010F00024030C94410880912503882319F0815022
:101100008093250360912103709122038091230332
:10111000909124030C94410870E00C942E1060917F
:1011200007018091210380FF0AC08091060123E01E
:10113000829FC00111248A5D9C4F0C948C08809181
:10114000080190910901891780F7E82FF0E09F01CD
:10115000220F331FE20FF31FEA5DFC4F1182108252
:1011600012828F5FF0CF9091210390FF16C0909173
:10117000080120910901921770F4E92FF0E0DF01D6
:10118000AA0FBB1FEA0FFB1FEA5DFC4F8183608340
:1011900042839F5FF0CF0C948F080895CF93DF9325
:1011A00000D01F92CDB7DEB79091210390FF0AC007
:1011B0009E012F5F3F4F0E941C084B8169818A81ED
:1011C0000E94B3080F900F900F90DF91CF91089578
:1011D000CF93DF93EC01EC81F0E0E550FD4F4491BB
:1011E000E1E2F3E0628181810E94CE088C818F5F11
:1011F0008C83DF91CF910895CF93DF93EC01E1E2EF
:10120000F3E0438162818C810E94CE088C818F5FE4
:101210008C83DF91CF9108950F931F93CF93DF932A
:1012200000D01F92CDB7DEB78C018091CF01811124
:101230000AC09E012F5F3F4F4FEF6FEF0E941C08C7
:101240008A818093CF01F8018481813051F028F0A8
:10125000823061F44091CF010AC08091CF0140E01B
:1012600007C06091CF0140E080E003C040E080E033
:1012700060E00E94B308F801848190E0019663E089
:1012800070E00E94ED2B84830F900F900F90DF9100
:10129000CF911F910F910895AF92BF92CF92DF929D
:1012A000EF92FF920F931F93CF93DF9300D01F9283
:1012B000CDB7DEB7182FF62E042FE22E9091210322
:1012C00090FF6DC0E92FE695AE2FB0E0A059BE4F5C
:1012D0008C91809329029E7F923061F49E012F5F52
:1012E0003F4F812F0E941C084B8169818A810E9497
:1012F000B30843C0823019F4009124033EC0863005
:1013000019F41091220339C08930D9F38931A9F534
:10131000E9518E2F8170D82EE695F0E0E550FC4F14
:10132000A590B490C12CBB2460910A01C61618F593
:101330002C2D30E0A29EC001A39E900DB29E900D78
:10134000112470E00E94D92B812FD11002C0860F8A
:1013500001C0861B90910801290F311DA901440F7E
:10136000551F240F351F2A5D3C4F402F6F2D0E94C3
:101370001C08C394D9CF0E948F0810932203F092C7
:10138000230300932403EE2051F060912103709118
:10139000220380912303909124030E9441080F901F
:1013A0000F900F90DF91CF911F910F91FF90EF90D1
:1013B000DF90CF90BF90AF900895E1E2F3E091818C
:1013C000282F4381628188E0890F0C944C0981E0C9
:1013D0000C94DD09E1E2F3E09181282F43816281E1
:1013E00088EF890F0C944C0981E00C94EA09E1E242
:1013F000F3E0628128E0620F08F46FEF282F438149
:1014000081810C944C0981E00C94F709E1E2F3E04E
:10141000628128E0621B08F460E0282F438181810B
:101420000C944C0981E00C94060AE1E2F3E043815C
:1014300028E0420F08F44FEF282F628181810C943D
:101440004C0981E00C94150AE1E2F3E0438128E0C5
:10145000421B08F440E0282F628181810C944C09E2
:1014600081E00C94240A20E00C944C09FF920F9325
:101470001F93CF93DF93EC01F12C0FEF10E06091FD
:101480000A01F616F0F4809108012F2D30E0280FA4
:10149000311DC901880F991F280F391F2A5D3C4F44
:1014A00070E0C8010E94ED2B962F8C81409124039F
:1014B00060912303F99E800D11240E941C08F3946F
:1014C000DECF0E948F089A818C8190FF02C08F5FCF
:1014D00001C081508C83DF91CF911F910F91FF90BC
:1014E0000895BF92CF92DF92EF92FF920F931F93D6
:1014F000CF93DF93FC01828180FF02C00FEF01C018
:1015000001E010E080910A01181708F040C08091B6
:101510000801C12ED12CE601C80FD11DCE01880FC4
:10152000991FC80FD91FCA5DDC4F198218821A8211
:1015300034E0E32EF12CB12C8091D1018B0D81315F
:1015400014F08F7005C087FF03C090910A01890FC6
:10155000082E000C990BC816D90691F4809124032B
:101560008E9DA0018F9D500D112455954795559541
:1015700047959E0160912303809122030E941C08DD
:10158000B00EF1E0EF1AF108B9F61F5FBBCF0E9471
:101590008F088091D101013031F4811102C0809116
:1015A0000A01815007C090E0019660910A0170E045
:1015B0000E94ED2B8093D101DF91CF911F910F916C
:1015C000FF90EF90DF90CF90BF900895CF938091E0
:1015D000080190910901891770F4E82FF0E09F014C
:1015E000220F331FE20FF31FEA5DFC4F11821082BE
:1015F00012828F5FF0CFC0E060910A01C617C0F57C
:10160000EC2FF0E070E0CF010E94ED2B209108015B
:10161000820F2091D001022E000C330B90E0E217D4
:10162000F307CCF020910501022E000C330B2E178E
:101630003F078CF09C01220F331F820F931F9C01E8
:101640002A5D3C4F40912403609123038091220343
:101650000E941C080BC0FC01EE0FFF1F8E0F9F1F86
:10166000FC01EA5DFC4F118210821282CF5FC4CF71
:101670000E948F08209104018091D001820F8093F5
:10168000D00190910501920F9093050119165CF419
:10169000082E000C990B40910A0150E0415051096D
:1016A000841795071CF0219520930401CF9108958C
:1016B0000F931F93CF93DF938C01FC01848195815D
:1016C00001968170992795838483C0E0D5E5809148
:1016D0000A01C81700F5809108012C2F30E0280F6F
:1016E000311DC901880F991F280F391F2A5D3C4FF2
:1016F0004C2F4695F80184819581840F911D81704E
:1017000040912403609123038D9F802D11240E941A
:101710001C08CF5FDCCFDF91CF911F910F910C940C
:101720008F080F931F93CF93DF93EC0100E010E03D
:1017300080910A01282F30E00217130724F59091B9
:1017400008019801290F311DA901440F551F240FCD
:10175000351F2A5D3C4F869590E04C81081719078C
:101760001CF4442331F002C0411103C04091240312
:1017700001C040E060912303809122030E941C0875
:101780000F5F1F4FD5CF0E948F088C8190E001968C
:10179000817099278C83DF91CF911F910F910895CC
:1017A0008F929F92AF92BF92CF92DF92EF92FF9271
:1017B0000F931F93CF93DF93FC01B280948081E05D
:1017C000848300E015E05BE4A52E88248394EE2456
:1017D000EA94F12C7BE4C72ED12C80910A010817E2
:1017E00008F08FC0C02FD0E01C9FF0011D9FF00DAE
:1017F0001124EE52FE4F911003C01382128267C073
:101800002381222389F1215023833481332319F04A
:101810009A2D921B01C0922F809124031C9FF001EE
:101820001D9FF00D1124EE52FE4F899FC00111241F
:10183000B6010E94D92B6283211104C0332311F019
:101840001482A38222E02B1508F441C01C9FF001F2
:101850001D9FF00D1124EE52FE4F809122038083D4
:1018600080912303818333C00E948F2C823091406A
:1018700074F582E08B1530F40E948F2CB7010E9422
:10188000ED2B02C0809122031C9FF0011D9FF00DE3
:101890001124EE52FE4F808322E02B1558F40E9453
:1018A0008F2C209123032695622F70E00E94ED2B50
:1018B000820F02C0809123031C9FF0011D9FF00D39
:1018C0001124EE52FE4F81831282A3828482809182
:1018D00008019E01280F311DC901880F991F280F8B
:1018E000391F2A5D3C4F1C9FF0011D9FF00D1124F4
:1018F000EE52FE4F4281618180810E941C080F5F81
:101900006CCFDF91CF911F910F91FF90EF90DF90FF
:10191000CF90BF90AF909F908F900C948F08E1E292
:10192000F3E080818E7F80836081718182819381E9
:101930000E94410810922A022FEF80E792E0215086
:1019400080409040E1F700C000000C948F08E1E275
:10195000F3E080818E7F808310922A022FEF80E750
:1019600092E0215080409040E1F700C000000C94CC
:101970008F0860912103669570E04BE050E08BE0AA
:1019800091E00E949F2C892B19F481E080932A0218
:101990000E94302090932302809322020895909118
:1019A000210390FF35C09170811102C0926006C082
:1019B0008B3210F0946502C0880F982B909321030E
:1019C000662351F0609121037091220380912303DB
:1019D000909124030E94410860912103669570E074
:1019E0004BE050E08BE091E00E949F2C892B19F096
:1019F00010922A0202C00E94B90C81E08093250255
:101A00004091240360912303809122030C94330AB4
:101A10000895682F90912103969581E0890F8B326C
:101A200008F081E00C94CF0C81E00C94090D682F34
:101A30009091210396958FEF890F09F48AE20C9417
:101A4000CF0C81E00C94170D61E00C94CF0CE1E217
:101A5000F3E080818160808386950C94240D8091D1
:101A6000210380FD0C948F0C0C94270D60E00C94E6
:101A7000CF0C8091280281112EC00E940F1E81116F
:101A800004C00E94C21E0E9453080E943D08609339
:101A900021037093220380932303909324036E7F8A
:101AA00061F40E9453080E943D08609321037093E3
:101AB000220380932303909324030E942A08109208
:101AC0002A028091210380FF03C086950E94360D73
:101AD00081E0809328020895E1E2F3E08081816053
:101AE000808386950C94360D10922A0208950F93E8
:101AF0001F93CF93DF9380912A02882309F49CC01F
:101B000080912902E0912103E695E81BE0932402ED
:101B1000823049F4F0E0E950FD4FE491CE2FD0E05F
:101B200008EE18E059C0863049F4F0E0EC50FD4F63
:101B3000E491CE2FD0E00CEF18E04EC0893051F484
:101B4000E695F0E0EF50FD4FE491CE2FD0E006E3B4
:101B50001AE042C08F3051F4E695F0E0E251FD4FBB
:101B6000E491CE2FD0E001E71AE036C0853149F488
:101B7000F0E0E551FD4FE491CE2FD0E006EE1AE003
:101B80002BC08831D9F0833239F4E9EEF2E0C59107
:101B9000D4910CE019E020C08432A9F08532C1F460
:101BA0008E2F63E00E94CD2BE92FF0E0EA51FD4F2C
:101BB000E491CE2FD0E000ED1BE00EC0C8EED3E0E4
:101BC00008E51BE009C0C4EFD1E001E91BE004C057
:101BD000C0EDD7E00BE118E080912502882389F061
:101BE000109225020E9430209E0120953095820F90
:101BF000931F909323028093220210922702109247
:101C0000260280912202909123020E943C208C1790
:101C10009D0790F0E0912202F0912302CE0FDF1F8A
:101C2000D0932302C093220282E292E0F801DF9176
:101C3000CF911F910F910994DF91CF911F910F9137
:101C40000895882311F0FA0101C0FB010994CF9394
:101C5000DF93C82FD62F0E9462088C1740F00E9495
:101C600062088D1720F4DF91CF910C94140D8C2F06
:101C7000DF91CF910C94240D0F931F93CF93FB0111
:101C8000C281CC2309F463C08C010E945E1D827264
:101C9000F801E25CFC45E431F10508F059C0EA5A6C
:101CA000FF4F0C94232C0E942F0D06C041E25DE0F3
:101CB00064E17DE00E94210EC0E04AC044E15DE0A5
:101CC00061E27DE0F7CF44EF59E067EE79E0F2CFD3
:101CD00047EE59E064EF79E0EDCF42E15AE063E08E
:101CE0007AE0E8CF43E05AE062E17AE0E3CF40E314
:101CF0005AE061E27AE0DECF41E25AE060E37AE066
:101D0000D9CF4BE758E06AE678E0D4CF4AE658E00E
:101D10006BE778E0CFCF81E017C065E082E010C0CC
:101D200068E086E00DC06EE089E00AC064E18FE003
:101D300007C067E185E104C088E106C062E289E18D
:101D40000E94270EB9CF83E20E94240DB5CFC1E0D7
:101D50008C2FCF911F910F9108950E940F1E81111A
:101D600002C00E94C21E0E944A1E80935603282F62
:101D700026952695269530E02630310524F087708B
:101D80008862809356038091560380FF04C0869535
:101D90008695869501C080E00C94BC0F2091560377
:101DA000822F869586958695482F50E045305105BF
:101DB00054F48F5F982F990F990F990F822F877086
:101DC000892B80935603809156038160809356033C
:101DD0000E944E1E809156038695869586950C949A
:101DE000BC0F80915603982F969596959695A1F0E5
:101DF000915E990F990F990F8770892B80935603E5
:101E0000887F91E009F490E08091560390FB80F97F
:101E1000809356030E944E1E8091560386958695A8
:101E200086950C94BC0F8091560380FD13C0816091
:101E300080935603813019F489E080935603809192
:101E400056030E944E1E8091560386958695869570
:101E50000C94BC0F08958091560380FF08C08E7FBC
:101E6000809356030E944E1E80E00C94BC0F089590
:101E70008091560380FD0C942B0F0C94130F9091BE
:101E80005603892F8695869586958F5F8F719770FB
:101E9000863038F4880F880F880F892B809356037B
:101EA00002C09093560380915603887F91E009F415
:101EB00090E08091560390FB80F9809356030E9436
:101EC0004E1E809156038695869586950C94BC0F80
:101ED000863008F085E0909156039770282F220FE6
:101EE000220F220F922B90935603987F21E009F442
:101EF00020E09091560320FB90F9909356030C94A8
:101F0000BC0F0E94680F809156030C944E1E9C01DA
:101F1000FB018281882349F12D3BFCE53F07C9F095
:101F200040F42B3BECE53E0769F02C3B3C4561F06F
:101F300008952F3B9CE5390791F070F0203C3C451B
:101F400089F0089585E001C080E00E94810F80E063
:101F500008950E94F10EFBCF0E94CE0EF8CF0E9492
:101F6000380FF5CF0E943F0FF2CF81E00895269AF7
:101F70002E9808952E980895CF92DF92EF92FF92B7
:101F8000CF93C82F863050F4811109C08091800012
:101F90008F7D809380000E94BA0F06C0C5E08091BB
:101FA00080008062809380002C2F30E0AFEFBFEF85
:101FB0000E94292C25E030E040E050E00E94012CF6
:101FC000C9012C3764E1360728F469E070E00E940B
:101FD000D92B29C0DA01C9018A50974DAF4FBF4FA5
:101FE0006627782F892F9A2F25EF38E241E050E0BD
:101FF0000E94012C69017A01CA01B9010E94BD2B1E
:102000009B01AC01C701B6010E94BD2BBB27A92FC4
:10201000982F872F009721E0A207B10511F0BC018E
:1020200002C06FEF7FEF70938B0060938A00CF91B7
:10203000FF90EF90DF90CF90089508950E94B70F22
:1020400082E28093800089E1809381008FEF9FEF8F
:1020500090938700809386000C94AD0E6A9A2EB1FF
:102060002B7F3EB134604FB7F894FC01CB01880F51
:10207000991F680F791F6E0F7F1FE617F70789F00A
:10208000819198E03EB9000000C087FF2EB9880F0B
:10209000000000C000C000C02EB900C09A9591F7A2
:1020A000ECCF4FBF8FE594E00197F1F700C000003F
:1020B00008950F931F93CF93DF93C62FD42F122F22
:1020C000FC0182818823C9F060932D020E94302098
:1020D00090932C0280932B0280E28C0F883008F0C2
:1020E00057C0C77081E001C0880FCA95EAF7DF9139
:1020F000CF911F910F910C94021580912D026813BE
:1021000030C080912B0290912C020E943C20883C90
:10211000910538F500E20D0FCD17B9F080E28C0F74
:10212000883040F4C77081E001C0880FCA95EAF793
:102130000E940915083028F581E09D2F977001C095
:10214000880F9A95EAF70E940215812F0E94EF14DA
:102150000830F0F4D77081E001C0880FDA95EAF713
:102160000AC080E28C0F883098F4C77081E001C00B
:10217000880FCA95EAF7DF91CF911F910F910C94C8
:102180000915812FDF91CF911F910F910C94EF14BE
:10219000DF91CF911F910F9108959C01CB01233FB7
:1021A0004CE53407F9F078F4283DFCE53F07B9F039
:1021B000293D4CE5340711F1273D3C4531F526E238
:1021C00041EE61EE1EC0253FFCE53F0799F070F03F
:1021D000263F3C45D1F427E245EE66EE12C027E2E9
:1021E00045EE0EC026E241EE60EE0BC027E245EE62
:1021F00064EE07C026E241EE62EE03C028E241E051
:1022000065EE0E94591080E00895FC0182818823C8
:1022100019F010922D02089581E00895CF93DF9375
:10222000EC01FB018281882309F41FC1C230FCE567
:10223000DF0708F41BC1C6319CE5D90738F09E01C1
:102240002A5F3C452930310508F010C10E942C1E40
:1022500090935C0380935B03C031ECE5DE0709F4E7
:10226000C3C008F041C0C8308CE5D80709F49AC053
:10227000F0F4C430ECE5DE0709F487C068F4C2303E
:102280008CE5D80709F477C0C330DC4509F0E3C01A
:1022900080915B03826076C0C630ECE5DE0709F40E
:1022A0006EC008F07BC080915B0388606BC0CC304F
:1022B0008CE5D80709F485C068F4CA30ECE5DE0780
:1022C00009F474C008F079C00E94921780915B03F2
:1022D000806858C0CE308CE5D80709F476C008F085
:1022E0007FC080915B038BC0CB3FECE5DE0709F438
:1022F0004FC018F5C3318CE5D80709F47DC078F4D8
:10230000C131ECE5DE0709F473C0C231DC4509F0E8
:10231000A2C00E94921780915B038F7733C0C531B2
:102320008CE5D80709F472C008F486C0CA3FDC45C2
:1023300009F091C080915C033EC0CF3FFCE5DF0710
:1023400009F45FC058F4CD3F9CE5D90709F444C0B7
:1023500008F43FC080915C0382602DC0C130FDE570
:10236000DF0709F475C008F45DC0C230DD4509F02F
:1023700072C080E06EC080915B03816003C0809179
:102380005B03806180935B0366C080915B0311C037
:1023900080915C03826080935C035DC080915B03ED
:1023A0008062F0CF80915B038064ECCF80915B030F
:1023B00088608460E7CF8160EECF80915B038E7F81
:1023C000E1CF80915B038D7FDDCF80915B03877FC1
:1023D000D9CF80915C0318C080915C038D7FDBCFE7
:1023E00080915B038F7ECECF80915B038F7DCACFC0
:1023F00080915B038F7BC6CF80915B03877F8B7F50
:10240000C1CF80915C038D7F8E7FC5CF80915B03B0
:1024100082FB222720F991E0922790FB82F990FB22
:1024200083F9B0CF80915C03982F909591708E7F47
:10243000892B90FB81F9AFCF0E94921780915B03AB
:1024400087FB222720F991E0922790FB87F99ACF0A
:1024500081E00E94C41E80915B0390915C030E9406
:102460003D1E0E94921780E001C081E0DF91CF9174
:102470000895CF93DF9386319C4541F5EB010E948F
:102480005E1D982F8A8120911601309117018823B3
:1024900079F09A7A81E009F480E080932E0291111C
:1024A00002C069E201C065E3C9010E945F1F0AC062
:1024B00080912E02811102C069E201C065E3C90169
:1024C0000E946A1F0E94AC1D80E001C081E0DF9184
:1024D000CF91089590933402809333020895E09150
:1024E0003302F0913402309721F00190F081E02D19
:1024F000099480E00895E0913302F091340230971E
:1025000099F020912A01222359F020915B0327FFA3
:1025100007C0DC012C9111962C93119725E02C9388
:102520000280F381E02D09940895E0913302F09147
:102530003402309739F022E0DC012C930480F581DD
:10254000E02D09940895209131023091320228172C
:10255000390771F09093320280933102E091330297
:10256000F0913402309721F00680F781E02D099434
:10257000089520912F02309130022817390771F009
:102580009093300280932F02E0913302F091340255
:10259000309721F00084F185E02D0994089585B7E6
:1025A000806885BF85B7806885BF089508950C94BD
:1025B000D6120C94D7120C94D6120C94D6120E94F8
:1025C000CF120E94DB120C94D91281E008950C9472
:1025D000E5120E9427200E9476060E94E1200E94B8
:1025E000AD0E0E94390D0C94DD127F928F929F9256
:1025F000AF92BF92CF92DF92EF92FF920F931F9311
:10260000CF93DF93CDB7DEB72A970FB6F894DEBF2E
:102610000FBECDBF0E94C8060E94E712811111C0F3
:102620008FEF89838A831B820E9430208160782FFC
:102630009D838C8349815A816B818D810E94A9136E
:102640004FC046E3A42E42E0B42E00E010E0702E0E
:10265000802F0E9461066C01F501819091905F01CD
:10266000882699268114910431F40F5F1F4F05309D
:10267000110569F7D5CF8091D80281FD0E946A06C5
:1026800080E0EE24E394F12C94012E213F21232BB2
:1026900009F18E837F82CE20DF2081E0CD2809F4EE
:1026A00080E088870E9430208160782F9A87898710
:1026B0004E815F8168858A850E94A913000F111FD2
:1026C000F801EA5CFD4F80819181E826F926F182CC
:1026D000E08206C08F5FEE0CFF1C8F30A9F6C5CFDD
:1026E0000E94770D0E941D100E9495230E946F1278
:1026F000909135028917C9F00E946F1280933502BC
:102700002A960FB6F894DEBF0FBECDBFDF91CF91F2
:102710001F910F91FF90EF90DF90CF90BF90AF90FF
:102720009F908F907F900C94F1032A960FB6F894A7
:10273000DEBF0FBECDBFDF91CF911F910F91FF90F4
:10274000EF90DF90CF90BF90AF909F908F907F9051
:102750000895CF93DF93CDB7DEB72B970FB6F894DC
:10276000DEBF0FBECDBF4F83588769877A878B87BF
:10277000DE01119686E0FD0111928A95E9F785E068
:10278000FE01379601900D928A95E1F749815A81B1
:102790006B817C818D819E810E944B1A2B960FB696
:1027A000F894DEBF0FBECDBFDF91CF910895FC013D
:1027B000808191810E941F1D0895CF93882309F481
:1027C000A4C0C82F8238C1F40E946F1281FD9DC041
:1027D00069E380911601909117010E945F1F0E948A
:1027E000AC1D2FEF81EE94E0215080409040E1F746
:1027F00000C0000069E319C0833801F50E946F1220
:1028000080FD83C063E580911601909117010E94BD
:102810005F1F0E94AC1D2FEF81EE94E0215080409D
:102820009040E1F700C0000063E5809116019091AF
:1028300017010E946A1FCF910C94AC1D8438C1F41B
:102840000E946F1282FD61C067E480911601909131
:1028500017010E945F1F0E94AC1D2FEF81EE94E0D4
:10286000215080409040E1F700C0000067E4DDCFD8
:102870008CEF8C0F813AD0F46C2F809116019091DF
:1028800017010E94DF1E882349F06C2F80911601EA
:10289000909117010E946A1F0E94AC1D6C2F8091BD
:1028A0001601909117010E945F1FC5CF80E28C0F27
:1028B000883048F4C77081E001C0880FCA95EAF7F4
:1028C0000E94611DB8CFEBE5EC0FE33040F4F0E07F
:1028D000E753FE4F808190E0CF910C94A312E8E57E
:1028E000EC0FE73150F4F0E0EE0FFF1FE556FE4F1E
:1028F00080819181CF910C94B912C03F30F08C2F20
:102900000E949D22CF910C948A23CF910895882311
:1029100009F464C0823879F40E946F1281FF5EC0AE
:1029200069E380911601909117010E945F1F0E9438
:10293000AC1D69E310C08338B1F40E946F1280FFB0
:102940004DC063E580911601909117010E945F1FB1
:102950000E94AC1D63E580911601909117010E94C1
:102960006A1F0C94AC1D843879F40E946F1282FFA8
:1029700035C067E480911601909117010E945F1F96
:102980000E94AC1D67E4E7CF9CEF980F913A10F4DA
:10299000682FE1CF90E2980F983050F4877091E063
:1029A00001C0990F8A95EAF7892F0E94671DD9CF38
:1029B0009BE5980F933020F480E090E00C94A312F4
:1029C00098E5980F973120F480E090E00C94B912CC
:1029D000803F20F00E9405230C948A230895CF9312
:1029E000C82F0E94DD13C93349F42FEF87EE93E01F
:1029F000215080409040E1F700C000008C2FCF9123
:102A00000C948714882321F00E94611D0C94AC1D46
:102A10000895882321F00E94671D0C94AC1D089531
:102A2000CF92DF92EF92FF920F931F93CF93DF939A
:102A30007C01062FC72FFC01158112951F70D281D2
:102A4000D1110E947E1D0E94571D882399F0DD231D
:102A500089F08C2F807F803421F080E2800F8830D5
:102A600048F082E00E94F61D0E94571D91E0D82E8A
:102A7000D92601C0D12CCC2EC2948FE0C8228C2D37
:102A800090E0FC01E659FF4F0C94232C8C2F807FA3
:102A9000CF70882311F0C295C07FDD2399F0CC233D
:102AA00009F48DC180E2800F883010F0011104C05C
:102AB0008C2F0E94611D03C08C2F0E94711D0E94EB
:102AC000AC1D7DC1802F0E948714CC2309F49CC1CA
:102AD00080E2800F883010F0011104C08C2F0E941A
:102AE000671D03C08C2F0E94771D0E94AC1D8CC1F6
:102AF0008C2F807FCF70803211F0C295C07F002371
:102B000019F00130C9F022C0DD2371F0112341F02A
:102B1000113031F40E94911D8C2B0E94991D74C1BB
:102B20000E94911D8C2B1DC0112319F0113009F446
:102B30006BC10E94A21D25C0DD2321F0163008F0D4
:102B400063C10EC0153008F05FC11BC0DD2361F00A
:102B5000112331F0F701858180FF31C18F708583AA
:102B60008C2F0E94021550C1112359F0093309F02E
:102B700037C1FFEF27EE83E0F15020408040E1F7BE
:102B80002DC18C2F0E9409153FC18C2F86958695EB
:102B9000837019F0813061F037C1DD2321F0802F7F
:102BA0009C2F937002C080E090E00E94A31234C179
:102BB000DD2321F0802F9C2F937002C080E090E0F5
:102BC0000E94B91229C1802FDD2319F00E949D2295
:102BD00002C00E9405230E948A231EC18C2F83708D
:102BE00009F045C0D11114C1402F42954695477058
:102BF000440F440F602F6F70862F90E0A0E0B0E08C
:102C0000042E04C0880F991FAA1FBB1F0A94D2F775
:102C100004FF10C00FE010E020E030E004C0000F1F
:102C2000111F221F331F4A95D2F70095109520954A
:102C3000309503C000E010E09801C695C695C370BA
:102C4000BC01CD01602B712B822B932BC23049F03C
:102C500058F4C13019F00E949C1BDAC00E948A1BF4
:102C6000D7C00E94AE1BD4C00E94881BD1C0DD23F8
:102C700019F08C2F817001C08695882309F4C8C093
:102C8000402F429546954770440F440F602F6F7058
:102C9000862F90E0A0E0B0E0042E04C0880F991FBA
:102CA000AA1FBB1F0A94D2F704FF10C00FE010E068
:102CB00020E030E004C0000F111F221F331F4A958F
:102CC000D2F7009510952095309503C000E010E0F4
:102CD0009801C695C695C370BC01CD01602B712BC0
:102CE000822B932BC23049F058F4C13019F00E9466
:102CF000611C8EC00E944F1C8BC00E94731C88C038
:102D00000E94C21B85C0CF70DD2339F08C2F0E943A
:102D1000E81B802F0E9402157BC0802F0E9409159E
:102D20008C2F0E94091C74C0023F01F128F4003F5F
:102D300041F0013FA1F03FC0033FF9F0043F39F1FA
:102D40003AC0DD2341F0153008F05EC08C2F8F7142
:102D50000E942E1C59C0163008F056C0F7CFDD2354
:102D600039F08C2F8F710E94E81B4EC0DD23C9F310
:102D70008C2F8F710E94091C47C0DD2329F08C2FF6
:102D80008F710E94D31B40C00E94CE1B3DC0DD232B
:102D900049F0CF718C2F0E94E81B63E08C2F0E94BA
:102DA000E11D32C081E00E94F61D123068F182E020
:102DB0000E94F61D29C0DD2331F0112391F2802FEE
:102DC0000E94DD1321C0112399F2093349F49FEFCA
:102DD000E7EEF3E09150E040F040E1F700C0000082
:102DE000802F0E94871410C04C2F4F70602FC70196
:102DF0000E9453040E94F91A0FC04C2F4F70602F8D
:102E0000C7010E94560408C088EF8C0D843020F45E
:102E10000E946F120E94F103DD20C9F00E94531D31
:102E200080FD15C0F70112820E944D1D0E94E81B13
:102E3000C7010E9448170E944D1DDF91CF911F913D
:102E40000F91FF90EF90DF90CF900C94091CDF91D1
:102E5000CF911F910F91FF90EF90DF90CF90089549
:102E60000F931F93CF93DF93EC01688179818A815F
:102E70000E942A1D8C010E94851C0E94761BB801AD
:102E8000CE010E941015DF91CF911F910F910895EF
:102E9000CF93DF93EC01988189812B813C81232B97
:102EA00031F08F3F31F481E09F3F19F403C081E09E
:102EB00001C080E080FD19C0CE010E940A0481118A
:102EC0000CC00E94571D882381F08A81882369F0F5
:102ED00082E0DF91CF910C94F61DCE010E94301755
:102EE000CE01DF91CF910C94D503DF91CF9108955E
:102EF0000E947E1D0E948E1D0E94AC1D0E94B42463
:102F00000E948A2380E090E00E94A31280E090E07B
:102F10000C94B91280911601909117010E94751FAF
:102F20000C9478170E946E1D0C948A17E92FE29575
:102F3000EF704E2F50E0FA013297EE30F105B0F409
:102F4000E658FF4F0C94232C803F91F018F4883EF4
:102F500068F40EC0843F51F40BC0883E48F0813FB6
:102F600029F406C093FB882780F9089580E008952E
:102F700081E008950E941F1D0E9496170895CF9327
:102F8000DF9300D000D01F92CDB7DEB70F900F9027
:102F90000F900F900F90DF91CF910895CF93DF9313
:102FA00000D000D000D0CDB7DEB726960FB6F8948B
:102FB000DEBF0FBECDBFDF91CF9108951F93CF939A
:102FC000DF93C091410216E080914202C81799F048
:102FD000D0E01C9FF0011D9FF00D1124ED5BFD4F13
:102FE0004081518162817381848195810E94CE17D5
:102FF0002196C770E9CFDF91CF911F91089540913D
:103000007302509174026091750270917602809102
:103010007702909178020C94CE170F931F93CF9361
:10302000DF938091780282958F7009F05DC0809166
:103030007502882309F458C0809141021091420220
:103040006091730270917402C0917602D091770200
:1030500091E06F3F09F090E0292F06E0811709F415
:1030600043C0209721F07F3F21F030E003C031E0E2
:1030700001C0322F90E030FD34C0089FF001099F5D
:10308000F00D1124DF01AD5BBD4F11963C911197FE
:10309000371327C03C91361324C012963C911297E7
:1030A00031111FC013964D915C9114974C1B5D0B11
:1030B000483C5105B0F4809178028F708061809314
:1030C0007802E85BFD4F80818F708061808383E7A9
:1030D00092E00E944817DF91CF911F910F910C94BD
:1030E000DE1701968770BACFDF91CF911F910F91B4
:1030F00008959F92AF92BF92CF92DF92EF92FF928C
:103100000F931F93CF93DF93CDB7DEB761970FB6C1
:10311000F894DEBF0FBECDBF8C0185E0F801DE0163
:103120001D9601900D928A95E1F7F8014081518139
:10313000E280909173026091740220917602309146
:1031400077022115310531F06F3F31F481E09F3F67
:1031500019F403C081E001C080E0F82FF1709F2EC8
:1031600080FD46C1F801A380B48083E7C82E82E0C9
:10317000D82EF0907502F501E21BF30BFF2009F445
:10318000DFC080917802E83CF10508F09BC0282F51
:10319000207F09F052C0561313C0491311C0FE2CF2
:1031A000E1100EC08F708061809378020E94FF173B
:1031B000C6010E94481780917802F801858358C1A2
:1031C000AB2831F05F3F31F481E04F3F19F403C089
:1031D00081E001C080E080FD03C081E08E2502C057
:1031E00080E090E0F82FF170FF2E80FF1CC08091EE
:1031F00041022091420236E0821709F417C190E0A3
:10320000389FF001399FF00D1124ED5BFD4F618176
:10321000561306C06081461303C06281E61203C0E4
:1032200001968770E9CFFE2CEE2009F421C1809130
:1032300078028160809378025AC0561306C0491301
:1032400004C0E11002C0F8019FC04D875E878D85E4
:103250009E850E94BA17882379F1EE2069F12091AA
:103260007802822F82958F7090E0029774F080919F
:1032700073029091740298878F831986BB86AA8601
:103280002C87CE0107960E94481786E0F801A3E735
:10329000B2E001900D928A95E1F70E940D180E940C
:1032A000FF170DC0561729F14D875E878D859E85C6
:1032B0000E94BA1781112CC0C8010E944817FF2430
:1032C000F394D6C0282F207F69F77A2DB98AA88A6F
:1032D0006E2D89890E94BF1783E792E00E944817EC
:1032E00086E0F60111928A95E9F70E94FF17F12C0A
:1032F000BFC04913D9CFE110D7CFF8018583C801EA
:103300000E94481786E0F60111928A95E9F7B0C04D
:10331000EE2091F220917802822F82958F7090E0BA
:1033200002970CF4B2CF80917302909174029A8349
:1033300089831B82BD82AC822E83CE010196A3CFEE
:10334000E83CF10508F047C0FE2CEE2009F4B4CFAC
:10335000561330C049132EC02091780220FD21C0A1
:10336000822F82958F70482F50E041155105C9F08A
:10337000F80125834F30510541F08F5F982F9295CA
:10338000907F822F8F70892B8583C8010E944817F8
:1033900086E0F801A3E7B2E001900D928A95E1F78B
:1033A00042C086E0F801A3E7B2E001900D928A9551
:1033B000E1F75EC04D875E878D859E850E94BA17B6
:1033C000811163CF80917802816080937802C80177
:1033D0000E9448174DC07A2DB98AA88A6E2D898916
:1033E0000E94BF1786E0F60111928A95E9F71BC08B
:1033F000EE2009F461CF4D875E878D859E850E9402
:10340000BA17F82E882309F457CF86E0F801A3E70E
:10341000B2E001900D928A95E1F783E792E00E9475
:10342000D7130E940D180E94FF1722C04D875E8798
:103430008D859E850E941F1D292F22952F70223079
:1034400028F49F7039F0811105C00BC0243028F496
:103450009F7049F4805E883020F0C8010E944817B0
:103460009F2CF92C05C0F8019581907F99F7F9CF31
:103470008F2D61960FB6F894DEBF0FBECDBFDF91E2
:10348000CF911F910F91FF90EF90DF90CF90BF9061
:10349000AF909F9008951F93CF93DF93CDB7DEB782
:1034A0002C970FB6F894DEBF0FBECDBF4F83588761
:1034B00069877A878B879C87CE0107960E94791847
:1034C0008823D1F09F8188852A853B85232B31F085
:1034D0008F3F31F481E09F3F19F403C081E001C0C8
:1034E00080E080FD47C04F81588569857A858B854E
:1034F0009C850E94CE173EC086E0FE013796DE0115
:10350000119601900D928A95E1F7FF81E8856A8511
:103510007B856115710531F0EF3F31F481E0FF3FAC
:1035200019F403C081E001C080E080FD23C0209138
:10353000420230E0C901019687709927409141020B
:1035400050E084179507F1F1F983EA837D836C835A
:1035500096E0929FD001939FB00D1124AD5BBD4FBB
:10356000FE01319601900D929A95E1F78093420207
:103570000E94DE1716E08091410290914202891765
:1035800071F1189FC00111248D5B9D4F0E94791825
:10359000882329F1E09141021E9FF0011124ED5B87
:1035A000FD4F4081518162817381848195810E94A8
:1035B000CE178091410290E0019687709927809301
:1035C0004102D9CF0E9492171092420210924102FA
:1035D000E3E7F2E086E0DF011D928A95E9F72C9699
:1035E0000FB6F894DEBF0FBECDBFDF91CF911F9114
:1035F0000895EF92FF920F931F93CF93DF938C0167
:10360000892B09F46CC0F12CEE24E394E801219697
:10361000F8018491843740F4843008F051C081303F
:1036200081F0823019F15BC0853709F444C0A8F1FC
:103630009CE7980F903708F052C08F770E9487144C
:1036400041C00E5F1F4FFE01849190E2980F9830A9
:1036500050F48770FE2D01C0FF0F8A95EAF78F2F77
:103660000E94811D14C00E94DD132DC00E5F1F4FEC
:10367000FE01849190E2980F983060F48770FE2DDF
:1036800001C0FF0F8A95EAF78F2F0E94871D0E94C5
:10369000AC1D19C00E94871416C00E5F1F4FFE019B
:1036A000C491CC2381F08FE99FE00197F1F700C02E
:1036B0000000C150F6CF0E5F1F4FFE01F49003C013
:1036C0000E94DD138E018F2D882309F49FCFEFE92F
:1036D000FFE03197F1F700C000008150F5CFDF9196
:1036E000CF911F910F91FF90EF9008950895089545
:1036F0000C94771B0C94781B0E947A1B6093AF028A
:103700007093B0028093B1029093B2020C94781738
:103710000C947C1B0F931F930091AF021091B00289
:103720002091B1023091B202602B712B822B932B2E
:103730001F910F910C947C1B0F931F930091AF026C
:103740001091B0022091B1023091B2026023712336
:10375000822393231F910F910C947C1B0F931F9333
:103760000091AF021091B0022091B1023091B202EB
:1037700060277127822793271F910F910C947C1B40
:103780000C94771B0E94C01B6093AB027093AC0239
:103790008093AD029093AE020C94781760E070E0D5
:1037A000CB010C94C21B0F931F9341E050E060E0EB
:1037B00070E08A019B0104C0000F111F221F331FFC
:1037C0008A95D2F7C901B8011F910F910C94C21BC1
:1037D0000F931F9341E050E060E070E004C0440F9D
:1037E000551F661F771F8A95D2F78091AB02909183
:1037F000AC02A091AD02B091AE028A019B01082BF0
:10380000192B2A2B3B2BC901B8011F910F910C9446
:10381000C21B0F931F9341E050E060E070E004C0D2
:10382000440F551F661F771F8A95D2F74095509514
:10383000609570958091AB029091AC02A091AD0221
:10384000B091AE028A019B01082319232A233B234E
:10385000C901B8011F910F910C94C21B0F931F93C4
:1038600041E050E060E070E004C0440F551F661F67
:10387000771F8A95D2F78091AB029091AC02A0910C
:10388000AD02B091AE028A019B01082719272A27B1
:103890003B27C901B8011F910F910C94C21B0F93D4
:1038A0001F930091AB021091AC022091AD023091B8
:1038B000AE02602B712B822B932B1F910F910C94D6
:1038C000C21B0F931F930091AB021091AC02209189
:1038D000AD023091AE0260237123822393231F91A6
:1038E0000F910C94C21B0F931F930091AB02109188
:1038F000AC022091AD023091AE0260277127822781
:1039000093271F910F910C94C21B08952FE0929F53
:10391000800D1124E82FE695E695E695877051E035
:1039200001C0550F8A95EAF785E0E89FF001112460
:10393000E758FD4F20E030E070E04081CB01022EDF
:1039400002C0969587950A94E2F781708195842745
:103950008523842781932F5F3F4F2530310569F7F9
:1039600008952FE0929F800D1124682F669566952B
:103970006695982F977085E0689FB001112440E00C
:1039800050E080E0FB01E40FF51FE758FD4F208178
:1039900030E0092E02C0369527950A94E2F721708F
:1039A0003327042E01C0220F0A94EAF7822B4F5FBF
:1039B0005F4F4530510531F70895BF92CF92DF92A6
:1039C000EF92FF920F931F93CF93DF938C01C090E0
:1039D000AB02D090AC02E090AD02F090AE028091CC
:1039E000AF029091B002A091B102B091B202C82A88
:1039F000D92AEA2AFB2ACFE1D0E0D701C6010C2E52
:103A000004C0B695A795979587950A94D2F780FD3F
:103A100004C0219790F7B12C07C0BC2EB8018C2FA1
:103A20000E9472040197A9F38B2DDF91CF911F9112
:103A30000F91FF90EF90DF90CF90BF900895CF93BC
:103A4000DF93EC010E94DD1CBE010E947204DF9135
:103A5000CF9108951F93CF93DF93EB019091400294
:103A6000992321F0CB010E941F1D13C0882349F028
:103A7000CB010E94DD1C182F682FCE010E94861CEE
:103A800004C0CB010E94B11C182FBE01812F0E94DF
:103A90007204DF91CF911F9108958091B3028595B3
:103AA0008595859508958091B302877008959091CA
:103AB000B302977081E009F480E008958091D70205
:103AC00008959091D702892B8093D702089580950D
:103AD0009091D70289238093D70208951092D7023C
:103AE00008959091D602892B8093D60208958095EF
:103AF0009091D60289238093D60208951092D6021F
:103B000008959091D502892B8093D50208958095D0
:103B10009091D50289238093D50208951092D50201
:103B200008958091B402089508950C94941D0C9406
:103B3000951D9091B402981721F08093B4020C94D3
:103B4000971D08958091B402882329F01092B40241
:103B500080E00C94971D0895E0911601F0911701F3
:103B60008091D7028083E0911601F0911701908136
:103B70008091D602892B8083E0911601F091170184
:103B800090818091D502892B80838091B402882313
:103B900081F0E0911601F09117019081892B8083CB
:103BA00080911601909117010E94C91E81110E94F7
:103BB000A21D80911601909117010C947B120C9418
:103BC000941D98E0899F90011124262B2093B30225
:103BD0000E94E81B8091B3028595859585950C948C
:103BE000DF1D1092B30280E00C94DF1D2091B30220
:103BF000809582238093B302982F977079F430E0F8
:103C0000482F082E000C550B2417350739F08595E1
:103C1000859585950E94091C0C94F11D089580E0FE
:103C200090E00E94BA2C21E08C3E9E4F09F020E0EB
:103C3000822F089582E090E00C94AC2C682F82E0F3
:103C400090E00C94C02C83E090E00C94AC2C682F96
:103C500083E090E00C94C02CCF9384E090E00E942D
:103C6000AC2CC82F81E290E00E94AC2C2C2F30E0CD
:103C7000A901582BCA01CF910895CF93C92F682F5E
:103C800084E090E00E94C02C6C2F81E290E0CF9104
:103C90000C94C02C86E090E00C94AC2C682F86E04D
:103CA00090E00C94C02CAB01BC018FE090E00C9430
:103CB000D22CAB01BC0183E190E00C94D22C60E0EB
:103CC00070E0CB010C94591E60E070E0CB010E94C3
:103CD000531E0C945F1E6CEE7EEF80E090E00E941D
:103CE000DE2C60E082E090E00E94C02C60E083E087
:103CF00090E00E94C02C1092AF021092B00210927D
:103D0000B1021092B20260E084E090E00E94C02C08
:103D100060E081E290E00E94C02C60E085E090E0ED
:103D20000E94C02C60E086E090E00E94C02C6FEF03
:103D300087E090E00E94C02C40E050E0BA0188E0AB
:103D400090E00E94D22C60E08DE090E00E94C02CB8
:103D500040E050E0BA0188E190E00E94D22C60E09F
:103D600087E190E00E94C02C40E050E0BA018CE175
:103D700090E00E94D22C60E080E290E00E94C02C93
:103D80000C94641E0C946B1E682F8EE090E00C94D3
:103D9000C02CFC01329680912A01882331F0809159
:103DA0005B0387FF02C09EE101C096E080E0915076
:103DB00028F021912223D9F38F5FF9CF089566234C
:103DC00051F120912A012223E9F020915B0327FF82
:103DD00019C0462F4695469546954E31E0F46770DA
:103DE00021E030E002C0220F331F6A95E2F7FC01A8
:103DF000E40FF11D828190E02823392381E0232BF9
:103E000069F409C0FC01329608962191621729F0E5
:103E1000E817F907D1F780E0089581E008959C0143
:103E2000FC0132969FEF80E04191461789F09F3F59
:103E300019F4411101C0982F8F5F8630A9F79F3F79
:103E400039F0F901E90FF11D97FDFA9562830895A4
:103E500008959C012A5F3F4FFC014281461301C037
:103E60001282019682179307B9F70895262F269597
:103E7000269526952E3168F4FC01E20FF11D67703E
:103E800021E030E001C0220F6A95EAF78281282BF9
:103E900022830895262F2695269526952E3170F497
:103EA000FC01E20FF11D677021E030E001C0220F3C
:103EB0006A95EAF72095828128232283089520912C
:103EC0002A01222329F020915B0327FD0C94361F41
:103ED0000C940F1F20912A01222329F020915B03CB
:103EE00027FD0C944A1F0C94291F20912A01FC01E4
:103EF0003296222331F080915B0387FF02C08EE16E
:103F000001C086E0DF011D928A95E9F708950895C2
:103F10000C94871F0C94871FCF930E948A1F0E94C6
:103F2000C8060E94881FC0E08C2F0E946106892B62
:103F300029F4CF5FC530C1F780E001C081E0CF91A7
:103F400008950C94871F0C94A11F0E94A31F8091B9
:103F50006103843009F43CC01092D90220E488E166
:103F600090E00FB6F894A895809360000FBE209360
:103F7000600080E00E94BC0F80E00E94F1030E947C
:103F8000740D8091DA0281110AC081E08093DA0217
:103F90008091210381708093DB020E94A70C0E9414
:103FA000A31F83B7817F846083BF83B7816083BF92
:103FB0007894889583B78E7F83BF0FB6F894A895C1
:103FC00080916000886180936000109260000FBE55
:103FD00008950C94871F0E9492170E94AD0E0E94B4
:103FE0006F120E94F1031092DA028091DB028111BC
:103FF0000E946C0D0E94B90C0C94E91F1F920F9245
:104000000FB60F9211248F939F93AF93BF9380911C
:10401000D902811113C08091570390915803A09148
:104020005903B0915A034196A11DB11D80935703C6
:1040300090935803A0935903B0935A03BF91AF9143
:104040009F918F910F900FBE0F901F90189582E057
:1040500084BD93E095BD9AEF97BD80936E0008955F
:104060002FB7F8948091570390915803A09159036A
:10407000B0915A032FBF08959C014FB7F8948091D7
:10408000570390915803A0915903B0915A034FBF21
:10409000821B930B089578941F920F920FB60F9284
:1040A00011248F939F93AF93BF9380915703909167
:1040B0005803A0915903B0915A030196A11DB11D57
:1040C0008093570390935803A0935903B0935A03D6
:1040D000BF91AF919F918F910F900FBE0F901F9046
:1040E000189581E08093E00080E28093D8001092E0
:1040F000C9008FE19EE40197F1F700C0000087E05E
:1041000090EBDC0180936A0390936B03A0936C03A4
:10411000B0936D039CE088E10FB6F894A895809366
:1041200060000FBE90936000FFCFAF92BF92CF921E
:10413000DF92EF92FF920F931F93CF93C0E0CC24B6
:10414000C394D12CE82EF12C8C2F0E9461065C01C7
:1041500000E010E0C601002E02C0880F991F0A94EB
:10416000E2F78A219B21892B31F40F5F1F4F0F301B
:10417000110581F70AC0602F7C2F80E00E94570450
:10418000E816F90691F781E004C0CF5FC530E1F68B
:1041900080E0CF911F910F91FF90EF90DF90CF9033
:1041A000BF90AF900895CF93C82F8CE20E949520C6
:1041B000882321F08C2FCF910C94952080E0CF9113
:1041C0000895CF930E940F1E811102C00E94C21E4B
:1041D000C5E6C15049F00E94C8068FE39CE90197EB
:1041E000F1F700C00000F5CF89E20E94D3208111D1
:1041F00020C18AE20E94D32081110E94C21E85E064
:104200000E94D32081110E9471200E941A1E809367
:10421000D80287E00E94D3208823A9F18BE10E9475
:10422000D320882351F08091D80281FB222720F9E6
:1042300091E0922790FB81F90EC08EE00E94D3207E
:10424000882361F08091D80282FB222720F991E037
:10425000922790FB82F98093D80215C080E10E94DA
:10426000D3209091D802882341F093FB222720F994
:1042700081E0822780FB93F904C0892F809580FB21
:1042800090F99093D8028091D8020E941E1E0E943D
:104290002C1E90935C0380935B0380EE0E94D320DE
:1042A000882341F080915B03982F909590FB80F9D3
:1042B00080935B0389E30E94D320882359F0809187
:1042C0005B0381FB222720F991E0922790FB81F983
:1042D00080935B0382EE0E94D320882359F0809163
:1042E0005B0382FB222720F991E0922790FB82F961
:1042F00080935B0386EE0E94D320882359F080913F
:104300005B0383FB222720F991E0922790FB83F93E
:1043100080935B0383EE0E94D320882359F0809121
:104320005B0384FB222720F991E0922790FB84F91C
:1043300080935B0385E30E94D320882359F080910A
:104340005B0385FB222720F991E0922790FB85F9FA
:1043500080935B0381E30E94D320882359F08091EE
:104360005B0386FB222720F991E0922790FB86F9D8
:1043700080935B0381E10E94D320882359F08091D0
:104380005B0387FB222720F991E0922790FB87F9B6
:1043900080935B0380915B0390915C030E943D1EC0
:1043A00087E20E94D320C82F8EE10E94D320811182
:1043B000C2608FE10E94D3208111C46080E20E941C
:1043C000D3208111C86081E20E94D3208111C06195
:1043D00082E20E94D3208111C06283E20E94D32036
:1043E0008111C06484E20E94D320882311F0C06848
:1043F00002C0CC2329F08C2F0E94271E6C2F03C0F3
:104400000E94231E682F70E080E090E00E94881BCD
:104410008FE00E94D320882319F081E00E94C41EFF
:1044200085E10E94D320882321F080E0CF910C9475
:10443000C41ECF9108958091E30280FF0BC060916C
:104440001D0185E0689FB0011124759567957595EC
:1044500067952BC081FF09C060911D0185E0689FB1
:10446000B00111247595679520C082FF07C0609147
:104470001D0185E0689FB001112417C09091E202F0
:104480009923D1F060911C01961788F720911D01A6
:1044900085E0289F90011124929FA001939F500DC9
:1044A000112470E0CA010E94ED2B6038710540F4C0
:1044B0006115710519F406C065E070E0862F089556
:1044C0008FE7089581E008958091E30280FF08C09E
:1044D0006091190170E0759567957595679521C094
:1044E00081FF06C06091190170E07595679519C04C
:1044F00082FF04C06091190170E010C09091E20247
:10450000992399F0609118019617A0F780911901ED
:10451000899FC001112470E00E94ED2B6038710565
:1045200040F46115710519F406C061E070E0862F52
:1045300008958FE7089581E00895803F21F40E9457
:104540001B22819504C0813F29F40E941B22809385
:10455000E7020895823F21F40E941B22819504C046
:10456000833F29F40E941B228093E6020895893F2D
:1045700019F40E94642205C08A3F31F40E9464222B
:1045800081958093E80208958B3F21F40E94642274
:10459000819504C08C3F29F40E9464228093E90233
:1045A0000895843F21F48091E502816017C0853F22
:1045B00021F48091E502826011C0863F21F4809150
:1045C000E50284600BC0873F21F48091E50288609A
:1045D00005C0883F31F48091E50280618093E50257
:1045E00008958D3F21F48091E30281600BC08E3FDE
:1045F00021F48091E302826005C08F3F29F480910D
:10460000E30284608093E3020895803F39F480914F
:10461000E70287FF6CC01092E70269C0813F29F46E
:104620008091E7021816BCF362C09091E602823FC7
:1046300029F497FF5CC01092E60259C0833F19F439
:104640001916CCF354C0893F41F48091E802181642
:104650000CF04DC01092E8024AC08A3F29F48091C4
:10466000E80287FF44C0F6CF8B3F39F48091E9021E
:1046700087FF3DC01092E9023AC08C3F29F4809137
:10468000E9021816BCF333C0843F21F48091E5029F
:104690008E7F17C0853F21F48091E5028D7F11C088
:1046A000863F21F48091E5028B7F0BC0873F21F488
:1046B0008091E502877F05C0883F31F48091E50253
:1046C0008F7E8093E50213C08D3F21F48091E30239
:1046D0008E7F0BC08E3F21F48091E3028D7F05C059
:1046E0008F3F29F48091E3028B7F8093E3028091D6
:1046F000E60281110EC08091E70281110AC080910B
:10470000E802811106C08091E902811102C0109275
:10471000E202089584EE92E00E9495120E943020F9
:104720009093E1028093E0020895CF93DF9300D04D
:1047300000D000D0CDB7DEB786E0E4EEF2E0DE01D7
:10474000119601900D928A95E1F78091E602811110
:1047500005C08091E702882309F47AC08091DE02C7
:104760009091DF020E943C20AC019091E2029923DB
:1047700039F020911E0130E02417350758F068C049
:1047800020911F018AE0289F9001112424173507EA
:1047900018F05EC09F3F19F09F5F9093E202109265
:1047A000E8021092E9028091E602181624F40E94B1
:1047B0001B228093E6028091E60287FF05C00E94DB
:1047C0001B2281958093E6028091E702181624F45B
:1047D0000E941B228093E7028091E70287FF05C0B9
:1047E0000E941B2281958093E7023091E6023323D9
:1047F000E1F02091E7022223C1F045EB3403C00130
:104800001124992319F09093E60203C081E080936C
:10481000E60235EB2303C0011124992319F090938C
:10482000E70203C081E08093E7020E948A2380911F
:10483000E0029091E1029093DF028093DE0286E035
:10484000FE013196A4EEB2E001900D928A95E1F757
:104850008091E802811105C08091E902882309F462
:104860007AC08091DC029091DD020E943C20AC0174
:104870009091E202992339F020911A0130E0241737
:10488000350758F068C020911B018AE0289F9001ED
:1048900011242417350718F05EC09F3F19F09F5F61
:1048A0009093E2021092E6021092E7028091E802F1
:1048B000181624F40E9464228093E8028091E80292
:1048C00087FF05C00E94642281958093E802809151
:1048D000E902181624F40E9464228093E902809170
:1048E000E90287FF05C00E94642281958093E90256
:1048F0003091E8023323E1F02091E9022223C1F054
:1049000045EB3403C0011124992319F09093E80278
:1049100003C081E08093E80235EB2303C00111243A
:10492000992319F09093E90203C081E08093E90292
:104930000E948A238091E0029091E1029093DD022F
:104940008093DC0286E0FE013196A4EEB2E0019095
:104950000D928A95E1F726960FB6F894DEBF0FBE4A
:10496000CDBFDF91CF910895E4EEF2E086E0DF0164
:104970001D928A95E9F71092E2021092E3020895DF
:1049800080910A030895CF93DF9300D01F92CDB793
:10499000DEB790916103943019F589837B836A8334
:1049A00082E08093E9008FEF9091E800815095FDBF
:1049B00006C095ED9A95F1F700008111F5CF809131
:1049C000E80085FF0DC040E050E063E070E0CE01FC
:1049D00001960E941F278091E8008E778093E8005F
:1049E0000F900F900F90DF91CF910895CF93DF93A9
:1049F000EC010E940227823011F0843031F4BE01B4
:104A000084E0DF91CF910C94C324DF91CF9108957E
:104A1000BC0183E00C94C324CF93DF93EC010E948C
:104A20000227823011F08430F9F482E08093E900AB
:104A30008FEF9091E800815095FD06C095ED9A9515
:104A4000F1F700008111F5CF8091E80085FF0CC0DF
:104A500040E050E066E070E0CE010E941F278091A8
:104A6000E8008E778093E800DF91CF910895CF938F
:104A7000DF93EC010E940227823011F08430D9F5D7
:104A800080912A01882339F080915B0387FF03C05E
:104A900060E282E002C068E081E08093E9008FEF8D
:104AA0009091E800815095FD06C095ED9A95F1F73B
:104AB00000008111F5CF8091E80085FF1CC0809136
:104AC0002A01811105C040E050E068E070E003C0B9
:104AD00070E040E050E0CE010E941F278091E80086
:104AE0008E778093E80080E2FE01AAEEB2E00190AA
:104AF0000D928A95E1F7DF91CF910895809160033F
:104B0000811109C00E94B0280E940D298091E20005
:104B100084608093E20008951092600308950895E0
:104B200008950C94EB1F42E061EC81E00E9429287B
:104B300042E261EC82E00C94292880916303833087
:104B400009F460C030F4813071F0823009F499C00A
:104B500008958A3009F485C08B3009F46BC0893020
:104B600009F0A7C020C080916203813A09F0A1C07A
:104B70008091E800877F8093E800809166039091A0
:104B80006703892B21F460E28AEE92E003C060E0C3
:104B900080E090E070E00E946A278091E8008B77C7
:104BA0008093E800089580916203813209F081C00A
:104BB0008091660390916703029708F07AC0809114
:104BC000E800877F8093E8008091E80082FD05C0BF
:104BD000809161038111F8CF6CC02091F300809126
:104BE000F20090E0922B029729F48091F1008B7FE4
:104BF000813021F48091F10080930A038091E800D4
:104C00008B7753C080916203813A09F052C0809142
:104C1000660390916703892B09F04BC08091E800EF
:104C2000877F8093E8008091E80080FFFCCF80912F
:104C30002A0136C0809162038132D9F580916603E2
:104C400090916703892BA9F58091E800877F809375
:104C5000E8000E945E288091640380932A010C94EE
:104C6000921780916203813221F58091E800877F5D
:104C70008093E8000E945E288091650380930B0377
:104C8000089580916203813AA1F48091E800877FC2
:104C90008093E8008091E80080FFFCCF80910B03B7
:104CA0008093F1008091E8008E778093E8000C9467
:104CB0005E28089584B7877F84BF0FB6F894A895BF
:104CC00080916000886180936000109260000FBE48
:104CD00090E080E80FB6F8948093610090936100B3
:104CE0000FBE0E94DF120E94B0280E940D29809101
:104CF000E20084608093E20078940E94A22B0E94DC
:104D0000E91280E291E00E946A128091610385308D
:104D100069F40E94A51F80915F038823B1F30E946C
:104D20008C1F882391F30E940927EFCF0E94F51270
:104D3000ECCF0C949B26292F332723303105C9F063
:104D400060F42130310581F02230310509F04AC08C
:104D50008BE390E028E235E049C02132310511F1C2
:104D60002232310579F13EC082E190E023E635E060
:104D70003DC099278130910561F040F08230910566
:104D800059F0039779F5E0E0F5E008C0E4E2F5E0DA
:104D900005C0E2E1F5E002C0E6E0F5E0849190E0D4
:104DA0009F0124C06115710541F061307105D1F496
:104DB00089E090E023E535E019C089E090E02AE33E
:104DC00035E014C06115710541F06130710551F491
:104DD0008CEB90E025E735E009C080E490E021E32A
:104DE00036E004C080E090E020E030E0FA0131835A
:104DF0002083089580916103843011F081E008954B
:104E000082E0089580910C03811102C00C94FA266F
:104E1000089580E189BD82E189BD09B400FEFDCF1E
:104E20008091D8008F7D8093D8008091E0008260CF
:104E30008093E0008091E00081FDFCCF0895CF9247
:104E4000DF92EF92FF920F931F93CF93DF93EC01CA
:104E50008B017A010E947D28811133C0E114F10495
:104E600039F0F70180819181081B190BC80FD91FF8
:104E7000C12CD12C0115110519F18091E80085FD97
:104E800016C08091E8008E778093E800E114F10469
:104E900049F0F70180819181C80ED91ED182C0826C
:104EA00085E00FC00E947D28882321F30AC08991E4
:104EB0008093F10001501109FFEFCF1ADF0ADACF1A
:104EC00080E0DF91CF911F910F91FF90EF90DF90E5
:104ED000CF90089520916803309169032617370712
:104EE00048F06115710539F42091E8002E77209380
:104EF000E80001C0B901FC0120E06115710579F1FC
:104F0000809161038823F1F18530F1F18091E8000F
:104F100083FD3CC08091E80082FD2EC08091E800B6
:104F200080FFEBCF2091F3008091F20090E0922B74
:104F30006115710551F08830910538F42191209365
:104F4000F100615071090196F3CF21E0089709F053
:104F500020E08091E8008E778093E800CECF211189
:104F6000CFCF0AC080916103882361F0853061F062
:104F70008091E80083FD0AC08091E80082FFF2CFB3
:104F800080E0089582E0089583E0089581E0089527
:104F900020916803309169032617370748F061159F
:104FA000710539F42091E8002E772093E80001C0C4
:104FB000B901FC0120E06115710591F18091610357
:104FC000882309F440C0853009F43FC08091E8008F
:104FD00083FD3DC08091E80082FD2FC08091E800F4
:104FE00080FFE9CF2091F3008091F20090E0922BB6
:104FF0006115710559F08830910540F42491209392
:10500000F1003196615071090196F2CF21E00897C5
:1050100009F020E08091E8008E778093E800CBCF04
:105020002111CCCF0AC080916103882361F08530C3
:1050300061F08091E80083FD0AC08091E80082FF62
:10504000F2CF80E0089582E0089583E0089581E042
:105050000895982F973068F59093E900981739F0E4
:105060007091EC002091ED005091F00003C0242FCE
:10507000762F50E021FD02C09F5FECCF3091EB0016
:105080003E7F3093EB003091ED003D7F3093ED009B
:105090003091EB0031603093EB007093EC00209383
:1050A000ED005093F0002091EE0027FDE5CF80E069
:1050B00008958F708093E90081E0089580916203E4
:1050C00087FF11C08091E80082FD05C080916103D7
:1050D0008111F8CF11C08091E8008B770BC08091CF
:1050E0006103882349F08091E80080FFF8CF809128
:1050F000E8008E778093E80008952091E4003091D5
:10510000E50095E64091EC00842F817040FF23C0BC
:105110008091E80080FD1DC080916103882399F093
:10512000853099F08091EB0085FD11C04091E4003D
:105130005091E5002417350729F3915011F09A0199
:10514000E1CF84E0089582E0089583E0089581E04E
:10515000089580E008954091E80042FFDDCF089572
:105160000E941E290E942629E0EEF0E080818160E5
:105170008083E8EDF0E080818F77808319BCA7ED14
:10518000B0E08C918E7F8C9380818F7E8083109293
:10519000600308950F931F93CF93DF930E941E29FE
:1051A0000E942629C8EDD0E088818F778883888186
:1051B0008068888388818F7D888319BC1092610301
:1051C00010925D0310925F0310925E0300EE10E0F8
:1051D000F80180818B7F808388818160888342E0B1
:1051E00060E080E00E942928E1EEF0E080818E7F7F
:1051F0008083E2EEF0E0808181608083808188603E
:105200008083F80180818E7F80838881806188839C
:10521000DF91CF911F910F910895E8EDF0E080812B
:105220008F7E8083E7EDF0E080818160808384E081
:1052300082BF81E0809360030C94CA28E8EDF0E01F
:1052400080818E7F80831092E20008951092DA00B0
:105250001092E10008951F920F920FB60F92112441
:105260002F933F934F935F936F937F938F939F936E
:10527000AF93BF93EF93FF938091E10082FF0BC048
:105280008091E20082FF07C08091E1008B7F8093D4
:10529000E1000E94A12B8091DA0080FF1FC0809165
:1052A000D80080FF1BC08091DA008E7F8093DA00E7
:1052B0008091D90080FF0DC080E189BD82E189BD68
:1052C00009B400FEFDCF81E0809361030E947E253A
:1052D00005C019BC109261030E948C258091E100E9
:1052E00080FF19C08091E20080FF15C08091E2002C
:1052F0008E7F8093E2008091E20080618093E200E3
:105300008091D80080628093D80019BC85E080939A
:1053100061030E9490258091E10084FF30C080915C
:10532000E20084FF2CC080E189BD82E189BD09B41F
:1053300000FEFDCF8091D8008F7D8093D8008091B2
:10534000E1008F7E8093E1008091E2008F7E809368
:10535000E2008091E20081608093E20080915D0331
:10536000882311F084E007C08091E30087FD02C02C
:1053700081E001C083E0809361030E9491258091C8
:10538000E10083FF29C08091E20083FF25C0809166
:10539000E100877F8093E10082E0809361031092B7
:1053A0005D038091E1008E7F8093E1008091E200B7
:1053B0008E7F8093E2008091E20080618093E20022
:1053C00042E060E080E00E9429288091F00088603F
:1053D0008093F0000E948F25FF91EF91BF91AF91D4
:1053E0009F918F917F916F915F914F913F912F91FD
:1053F0000F900FBE0F901F9018951F920F920FB62F
:105400000F9211242F933F934F935F936F937F934A
:105410008F939F93AF93BF93CF93DF93EF93FF93BC
:10542000C091E900CF708091EC00D82FD17080FD41
:10543000D0E81092E9008091F000877F8093F0001F
:1054400078940E94412A1092E9008091F0008860CF
:105450008093F000CD2BCF70C093E900FF91EF91C6
:10546000DF91CF91BF91AF919F918F917F916F917C
:105470005F914F913F912F910F900FBE0F901F9012
:1054800018951F93CF93DF93CDB7DEB7AA970FB6CA
:10549000F894DEBF0FBECDBFE2E6F3E08091F100ED
:1054A000819323E0EA36F207C9F70E949D25809197
:1054B000E80083FF2EC18091620390916303492F1E
:1054C00050E04A30510508F024C1FA01E857FF4F77
:1054D0000C94232C803821F0823809F01AC108C0BE
:1054E00080915E0390915F03992389F082600FC0E1
:1054F000809166038F70873008F00BC18093E900BC
:105500008091EB0085FB882780F91092E90090914B
:10551000E800977F9093E8008093F1001092F100EB
:10552000D1C0282F2D7F09F0F4C0882319F08230D4
:1055300061F0EFC080916403813009F0EAC09330DC
:1055400009F080E080935F032EC080916403811195
:105550002AC0809166038F702FEF280F263008F045
:10556000D8C08093E9002091EB0020FF1CC093304D
:1055700021F48091EB00806214C09091EB00906167
:105580009093EB0021E030E0A90102C0440F551FC9
:105590008A95E2F74093EA001092EA008091EB00CE
:1055A00088608093EB001092E9008091E800877F8B
:1055B0008093E8000E945E28ACC08111AAC01091BF
:1055C00064031F778091E3008078812B8093E30050
:1055D0008091E800877F8093E8000E945E28809198
:1055E000E80080FFFCCF8091E30080688093E300B7
:1055F000111102C082E001C083E08093610389C081
:105600008058823008F085C08091640390916503D2
:105610008C3D53E0950779F583E08A838AE289839C
:105620004FB7F894DE01139620E03EE051E2E32FFD
:10563000F0E050935700E49120FF03C0E295EF7033
:105640003F5FEF708E2F90E0EA3010F0C79601C0F8
:10565000C0968D939D932F5F243149F74FBF809162
:10566000E800877F8093E8006AE270E0CE0101964F
:105670000E946A2716C06091660370916703AE01AD
:105680004F5F5F4F0E949926BC01892B09F441C0EE
:105690009091E800977F9093E80089819A810E9419
:1056A000C8278091E8008B778093E80032C080386B
:1056B00081F58091E800877F8093E80080915D0309
:1056C0008093F1008091E8008E7772CF811121C024
:1056D000809164039091650399270297D4F4809197
:1056E000E800877F8093E8008091640380935D03E6
:1056F0000E945E2880915D03811106C08091E300C5
:1057000087FD02C081E001C084E0809361030E94B4
:1057100093258091E80083FF0AC08091E800877F8D
:105720008093E8008091EB0080628093EB00AA9662
:105730000FB6F894DEBF0FBECDBFDF91CF911F91A2
:1057400008950895CF93809161038823A1F0C091BB
:10575000E900CF709091EC00892F817090FD80E876
:10576000C82B1092E9008091E80083FD0E94412A35
:10577000CF70C093E900CF910895DB018F939F9381
:105780000E94382CBF91AF91A29F800D911DA39FC5
:10579000900DB29F900D11240895991B79E004C0DB
:1057A000991F961708F0961B881F7A95C9F7809560
:1057B0000895AA1BBB1B51E107C0AA1FBB1FA61758
:1057C000B70710F0A61BB70B881F991F5A95A9F7AA
:1057D00080959095BC01CD01089597FB072E16F496
:1057E000009407D077FD09D00E94D92B07FC05D083
:1057F0003EF4909581959F4F0895709561957F4FE8
:105800000895A1E21A2EAA1BBB1BFD010DC0AA1F01
:10581000BB1FEE1FFF1FA217B307E407F50720F019
:10582000A21BB30BE40BF50B661F771F881F991F94
:105830001A9469F760957095809590959B01AC01DD
:10584000BD01CF010895EE0FFF1F0590F491E02DEB
:105850000994A29FB001B39FC001A39F700D811D49
:105860001124911DB29F700D811D1124911D089569
:105870000E94292CA59F900DB49F900DA49F800D90
:10588000911D112408958F929F92AF92BF92CF9253
:10589000DF92EF92FF92CF93DF93EC0168817981E1
:1058A0008A819B81611571058105910521F464E26E
:1058B00079ED8BE597E02DE133EF41E050E00E9478
:1058C000F42C49015A019B01AC01A7EAB1E40E9402
:1058D000382C6B017C01ACEEB4EFA50194010E9461
:1058E000162DDC01CB018C0D9D1DAE1DBF1DB7FF1C
:1058F00003C00197A109B04888839983AA83BB8319
:105900009F77DF91CF91FF90EF90DF90CF90BF9086
:10591000AF909F908F9008950E94432C089580E04F
:1059200091E00E94432C0895A0E0B0E08093000134
:1059300090930101A0930201B09303010895FC012B
:105940004150504030F001900616D1F73197CF0109
:105950000895882799270895F999FECF92BD81BDB2
:10596000F89A992780B50895A6E1B0E044E050E0A8
:105970000C94E62CA8E1B0E042E050E00C94E62C58
:10598000262FF999FECF92BD81BDF89A019700B4F8
:10599000021639F01FBA20BD0FB6F894FA9AF99A98
:1059A0000FBE08950396272F0E94C12C0E94C02C81
:1059B000252F0E94C12C242F0C94C12C0196272F37
:1059C0000E94C12C0C94C02CDC01CB01FC01F99984
:1059D000FECF06C0F2BDE1BDF89A319600B40D923B
:1059E00041505040B8F70895052E97FB1EF40094DF
:1059F0000E940B2D57FD07D00E94012C07FC03D0FD
:105A00004EF40C940B2D50954095309521953F4FB9
:105A10004F4F5F4F089590958095709561957F4F9A
:105A20008F4F9F4F0895B7FF0C94382C0E94382C4D
:0A5A3000821B930B0895F894FFCF3A
:105A3A00010000000102001000101001191A1B1CBD
:105A4A001D1E1F202122B5022808641E140A321EB8
:105A5A00C02437250C250825F62401E200E900EACE
:105A6A0000B500B600B700CD008301CC008A0192D0
:105A7A000194012102230224022502260227022A76
:105A8A0002B300B4006F007000818283F0F1C66730
:105A9A0066379431303534979633F49091929395D2
:105AAA000001020202020606060909090909090F8C
:105ABA000F0F0F0F0F15151518191919191919198B
:105ACA001919192324252525252525E200E900EAA7
:105ADA0000B500B600B700CD008301CC008A019260
:105AEA000194012102230224022502260227022A06
:0C5AFA0002B300B4006F007000818283D2
:00000001FF
